:020000040800F2
:10000000300B0020CD010008771B0008A118000864
:10001000751B0008FB020008092200080000000010
:10002000000000000000000000000000391C000873
:100030002503000800000000791B00082D1F0008A0
:10004000E7010008E7010008E7010008E7010008F0
:10005000E7010008E7010008E7010008E7010008E0
:10006000E7010008E7010008E7010008E7010008D0
:10007000E7010008E7010008E7010008E7010008C0
:10008000E7010008E7010008E7010008E7010008B0
:10009000E7010008E7010008E7010008E7010008A0
:1000A000E7010008E7010008E7010008E701000890
:1000B000E7010008E7010008E7010008E701000880
:1000C000E7010008E7010008E7010008E701000870
:1000D000E7010008E7010008E7010008DD2100084A
:1000E000E7010008E7010008E7010008E701000850
:1000F000E7010008E7010008E7010008E701000840
:10010000E7010008E7010008E7010008E70100082F
:10011000E7010008E7010008E7010008E70100081F
:10012000E7010008E7010008E7010008E70100080F
:1001300000F002F800F03AF80AA090E8000C8244BF
:100140008344AAF10107DA4501D100F02FF8AFF29C
:10015000090EBAE80F0013F0010F18BFFB1A43F0A5
:1001600001031847B4250000D4250000103A24BF2D
:1001700078C878C1FAD8520724BF30C830C144BF0C
:1001800004680C607047000000230024002500264E
:10019000103A28BF78C1FBD8520728BF30C148BFEA
:1001A0000B6070471FB51FBD10B510BD00F06BF898
:1001B0001146FFF7F7FF02F05FFA00F089F803B489
:1001C000FFF7F2FF03BC00F091F8000009488047F8
:1001D00009480047FEE7FEE7FEE7FEE7FEE7FEE729
:1001E000FEE7FEE7FEE7FEE704480549054A064B41
:1001F000704700008F1F0008310100083005002003
:10020000300B00203007002030070020B2F120031F
:100210000AD5C2F1200320FA02F001FA03F321FA11
:1002200002F140EA0300704721FA03F04FF00001A9
:1002300070474FF0000200B51346944696462039A9
:1002400022BFA0E80C50A0E80C50B1F12001BFF48F
:10025000F7AF090728BFA0E80C5048BF0CC05DF8F5
:1002600004EB890028BF40F8042B08BF704748BF43
:1002700020F8022B11F0804F18BF00F8012B7047B7
:10028000704770477047754600F02CF8AE46050081
:100290006946534620F00700854618B020B5FFF7A1
:1002A000A3FFBDE820404FF000064FF000074FF0DD
:1002B00000084FF0000B21F00701AC46ACE8C00984
:1002C000ACE8C009ACE8C009ACE8C0098D4670478D
:1002D00010B50446AFF300802046BDE81040FFF79C
:1002E0006EBF000000487047D0040020014918206C
:1002F000ABBEFEE7260002007047FEE730B50446BD
:100300000020651804E000BF14F8011B01F06CFF29
:10031000AC42F9D3002101F067FFBDE83040002175
:1003200001F062BF704772B6FEE7000030B585B0DD
:1003300000250446049500F01FFC0A480121001B1B
:10034000C00A03900095CDE9011404A9684600F0A5
:10035000C1FA044600F0B2FB14B1012005B030BD73
:100360000020FBE70000050800B587B000F004FCA2
:10037000684600F02DFB00F0A1FB0348029988437A
:1003800000D0022007B000BDF0FF0F0010B500F054
:10039000F3FB03493420C860BDE8104000F08EBB79
:1003A000002002402DE9F04116468846054600240B
:1003B00000F0E2FB0E4F13E058F8242000232946FA
:1003C000022000F099FB10B10320BDE8F08158F83D
:1003D00024002968814201D00220F6E7641C2D1D0B
:1003E000B44201D2BD42E7D900F068FB0020ECE73F
:1003F000FCFF040810B58EB0044607A800F0E8FA28
:10040000ACB10020019001200090A5208DF81000D3
:100410009DF82D008DF811000A48099C044300F056
:10042000ABFB00F057FB00F0A9FA10B107E0012088
:10043000E8E76846029400F0DDFA002800D00420C6
:100440000EB010BDF0FF0F0006490020C86106483D
:10045000016941F004010161016941F0400101615C
:1004600070470000B0040020002002402DE9F04752
:10047000DFF89C80D8F820104CF250390143CFB2FD
:10048000C1F30726C1F307450C0E484600F02AF9D0
:1004900000283BD11F49C86100F070FA002835D10F
:1004A000D8F8102042F01002C8F81020FF2F07D013
:1004B0001948018839430180484600F013F9F8B91A
:1004C000FF2E08D01448801C018831430180484623
:1004D00000F008F9A0B9FF2D08D00F48001D0188D1
:1004E00029430180484600F0FDF848B9FF2C07D0A9
:1004F0000948801D018821430180484600F0F2F838
:10050000D8F8102022F01002C8F81020BDE8F087BB
:1005100000200240B004002008F8FF1F2DE9F0473A
:10052000DFF89C80D8F820104CF250398143CFB2CC
:10053000C1F30726C1F307450C0E484600F0D2F878
:1005400000283BD11F49C86100F018FA002835D1B6
:10055000D8F8102042F01002C8F81020FF2F07D062
:100560001948018839400180484600F0BBF8F8B9C5
:10057000FF2E08D01448801C018831400180484675
:1005800000F0B0F8A0B9FF2D08D00F48001D018879
:1005900029400180484600F0A5F848B9FF2C07D053
:1005A0000948801D018821400180484600F09AF8E2
:1005B000D8F8102022F01002C8F81020BDE8F0870B
:1005C00000200240B004002008F8FF1F0449A520C5
:1005D000C96901F00201022900D100207047000022
:1005E0000020024070B506464CF25035284600F017
:1005F00079F8002820D11149C861114C206940F0D8
:1006000020002061206940F040002061284600F071
:1006100069F8216921F02001216100280CD12069AD
:1006200040F01000206107480680284600F05AF884
:10063000216921F01001216170BD0000B00400208B
:100640000020024000F8FF1F064A0021D161064940
:100650000A6942F002020A614861086940F04000FC
:1006600008617047B004002000200240044B0022C3
:10067000DA61044A136943F0010313610180704792
:10068000B00400200020024014480022C168CB06BC
:10069000134904D5CA6942F00202CA611022C36834
:1006A0005B0705D5CB6943F00103CB6142F004023F
:1006B000C369DB0707D0CB6943F00403CB61C16991
:1006C00021F00101C161A2F58071013901D0C26040
:1006D0007047C16921F00101C161704700200240EB
:1006E000B004002070B5054600F056FB0646114CDC
:1006F00009E0681C07D025B100F04EFB801BA84222
:1007000001D9032070BDE068C007F2D1E06880061F
:1007100001D52020E060E068C00605D4E069C0078C
:1007200002D1E068400703D5FFF7AEFF012070BD9E
:10073000002070BD0020024010B590F8211000226A
:10074000022905D00421816380F82020012010BDFA
:1007500001680B6823F00E030B6001680B6823F03F
:1007600001030B6090F84030C46B012101FA03F3E0
:10077000636080F8211080F82020104610BD000032
:100780002DE9F05F90F821100024022903D0042104
:100790008163012485E001680A6822F00E020A6084
:1007A00001680A6822F001020A603F4E3E4FB2150E
:1007B000DFF8F4C0DFF8F090DFF8ECA0DFF8E8B085
:1007C000DFF8E4E00168783F13011502ACF1640C36
:1007D000A9F15009AAF13C0AABF1280BAEF1140EB5
:1007E0004FF48018B14227D9B9420ED0614512D0DA
:1007F00049451DD0514518D0594518D0714501D1F2
:10080000424615E0294EB14201D1012210E0274EA7
:100810001436B14201D110220AE0244E2836B142EA
:1008200006D0224A3C32914201D11A4600E02A46C3
:100830001E49091F0A602BE0B94213D0614517D049
:10084000494522D051451DD059451DD0714501D192
:1008500042461AE0B14202D14FF0807215E0134EC9
:10086000B14201D1012210E0104E1436B14201D143
:1008700010220AE00D4E2836B14206D00B4A3C3217
:10088000914201D11A4600E02A46074980394A6060
:10089000012180F82110002180F82010416B01B166
:1008A00088472046BDE8F09F8000024008040240CF
:1008B00070B5044600F070FA0546601C02D004488A
:1008C0000078044400F068FA401BA042FAD370BDDF
:1008D000100000202DE9F047054626480F46012666
:1008E000017E01290FD00121814601762868DFF8B9
:1008F00088804CF25034022808D0A2462046FFF7E8
:10090000F1FEA8B131E00220BDE8F0872046FFF7F4
:10091000E9FE08BB0120FFF797FD2046FFF7E2FE46
:10092000D8F81010064621F00401C8F810101CE099
:100930004FF0FF303860AC6811E02046FFF784FECE
:100940005046FFF7CFFED8F81010060021F0020144
:10095000C8F8101001D03C6007E004F50064D5E948
:10096000020100EBC120A042E7D8002189F818104D
:100970003046C9E7B00400200020024070B5FFF700
:1009800025FEC5B24CF250363046FFF7ABFE0028CC
:1009900018D10D49C8610D4C206940F0200020613C
:1009A000206940F0400020613046FFF79BFE21693E
:1009B00021F020012161002804D12846BDE87040C3
:1009C000FFF710BE70BD0000B00400200020024000
:1009D00070B50446064D07202060286AA060FFF726
:1009E000F5FD2074E869C0F38200607470BD0000FA
:1009F000002002402DE9F0472D4D04460120297EBC
:100A000001290ED00121297621784FF00007C9076E
:100A10000DD060680128A06806D0FFF727FDE8BB6D
:100A200005E00220BDE8F087FFF778FDF7E72178C1
:100A3000890703D5207CFFF7D5FD78BB21781D4EB3
:100A400049074CF2503916D594F811804846FFF703
:100A500049FE78B9EF61306940F010003061164905
:100A600048F0880008804846FFF73CFE316921F0D5
:100A70001001316190B92178090716D5D4F8148096
:100A8000247E4846FFF72EFE40B9EF61306940F002
:100A900010003061A8F80040484600E005E0FFF78C
:100AA00021FE316921F0100131612F76BAE7000093
:100AB000B00400200020024002F8FF1F0348016933
:100AC00041F08001016100207047000000200240D9
:100AD00000F000BA05480169890505D40449816020
:100AE00004498160002070470120704700200240C7
:100AF00023016745AB89EFCD2DE9F05F07461C4820
:100B000088460024017E15461E46012909D0012190
:100B1000814601764CF2503A5046FFF7E3FD18B19A
:100B200022E00220BDE8F09F012F02D0022F00D06A
:100B30000427D346DFF83CA0220128463146FFF7C0
:100B400065FB81B208EB4400FFF790FD5846FFF7C4
:100B5000C9FDDAF8102022F00102CAF8102018B9F5
:100B6000641CE4B2BC42E7D3002289F81820D9E71C
:100B7000B004002000200240064900200A69120645
:100B800007D5054A4A60054A4A600969090600D541
:100B9000012070470020024023016745AB89EFCD5B
:100BA0002DE9F84FDFF8C8910024A9F1040B234682
:100BB0000F2709F1040AABF1040ED1E00125A5408D
:100BC00006EA0502AA4276D1DFF8A8C14E68A6EB74
:100BD0000C0866452BD00DDC032E34D005DC36B373
:100BE000012E19D0022E2FD11BE0112E16D0122E5D
:100BF0002AD119E0B8F5881F19D006DCB8F5803F76
:100C000015D0B8F5801F1FD111E0B8F5001F0ED028
:100C1000B8F5041F18D10AE0CB6815E0CB681B1D9E
:100C200012E0CB6808330FE0CB680C330CE08B6824
:100C30002BB1012B4FF0080303D0456104E00423DE
:100C400002E0056100E00023FF2A01D8064601E02A
:100C500000F104064FEA840501D9A5F12005D6F874
:100C6000008007FA05FC28EA0C0803FA05F548EAB3
:100C70000508C6F800804D68ED0070D53E4DAE69A0
:100C800046F00106AE61AD6924F0030605F00105EA
:100C900000953A4D06EB050CDCF80850A607360F18
:100CA00007FA06F825EA0805DFF8D480404503D1A5
:100CB0004FF0000825E052E0DFF8C880404502D13F
:100CC0004FF001081DE0DFF8C080404502D14FF031
:100CD000020816E0DFF8B480404502D14FF0030867
:100CE0000FE0DFF8AC80404502D14FF0040808E087
:100CF000DFF8A080404502D14FF0050801E04FF039
:100D0000060808FA06F848EA0508CCF808804D6895
:100D1000D9F80060ED024D4601D5164300E0964338
:100D20002E604D68DAF80060AD02554601D51643D5
:100D300000E096432E604D68DBF80060AD035D4631
:100D400001D5164300E096432E604D68DEF8006042
:100D5000ED03754601D5164300E096432E60641CF2
:100D60000A681646E2407FF429AFBDE8F88F00001C
:100D70000804014000001110001002400000014072
:100D800000080140000C0140001001400014014027
:100D900000180140001C01400148806870470000B5
:100DA0001000002002488168027811448160704779
:100DB00010000020074810B5016841F010010160E3
:100DC000032000F075F80F2000F006F800F024F87A
:100DD000002010BD0020024070B50D4D04464FF4B8
:100DE0007A712878B1FBF0F00A490968B1FBF0F09C
:100DF00000F0EEFA48B9102C07D200222146501E0E
:100E000000F036F800206C6070BD012070BD00005D
:100E1000100000201C0000200C4808B5816941F03A
:100E200001018161816901F001010091C16941F015
:100E30008051C161C06900F0805000900448416851
:100E400021F0E06141F00071416008BD00100240F6
:100E500000000140002809DB00F01F020121914041
:100E60004009800000F1E020C0F800117047000048
:100E7000F0B40E4B1B680C46C3F30223C3F1070505
:100E8000042D00D90425191D072901D2002300E0F3
:100E9000DB1E012606FA05F1491E214099409E40BD
:100EA000761E16403143F0BC01F0D6BB0CED00E0DD
:100EB000064900F0070208684FF6FF03184040EAB1
:100EC0000220034A10430860704700000CED00E068
:100ED0000000FA05BFF34F8F05480168054A01F489
:100EE000E06111430160BFF34F8F00BFFDE70000D9
:100EF0000CED00E00400FA052DE9F0470F4605006F
:100F000061D0434E306800F00700B84209D2306823
:100F100020F0070038433060306800F00700B84226
:100F200051D128683B4C810712D5400703D5606832
:100F300040F4E06060602878000703D5606840F402
:100F4000605060606068A96820F0F000084360604D
:100F50002878C00728D06868012810D021680228A6
:100F600010D0890700292EDA616821F003010143BE
:100F70006160FFF711FF804641F288390DE021687A
:100F80008903EFE78901EDE7FFF706FFA0EB080112
:100F9000494502D90320BDE8F0876068696800F020
:100FA0000C00B0EB810FEFD1306800F00700B842C1
:100FB0000BD9306820F0070038433060306800F00B
:100FC0000700B84201D00120E5E72878400705D5A1
:100FD0006068E96820F4E0600843606028780007F2
:100FE00006D56068296920F4605040EAC10060605D
:100FF00000F038F86168084AC1F30311515CC84039
:101000000649086006480068FFF7E6FE0020C2E7D0
:101010000020024000100240AC2600081C00002006
:10102000140000200448054900684968044AC1F3D7
:101030000221515CC84070471C0000200010024093
:10104000BC2600080448054900684968044AC1F301
:10105000C221515CC84070471C00002000100240B3
:10106000BC2600080E4A51680E4801F00C03042B00
:1010700011D0082B0FD10C48C1F38343C903C05CC6
:101080000AD55168084AC1F34041921E515C054A95
:101090005043B0FBF1F070470449484370470000EB
:1010A0000010024000127A009C26000800093D0052
:1010B0002DE9F84F040070D02078C04DC00749D00A
:1010C0006868C0F38100012807D06868C0F3810018
:1010D000022809D16868C00306D52868800339D57D
:1010E00060680028E7D035E06068B0F5803F0BD03D
:1010F00010B1B0F5A02F11D0286820F480302860FE
:10110000286820F4802002E0286840F480302860BD
:10111000606890B1FFF740FE06460AE0286840F498
:1011200080202860F0E700BFFFF736FE801B6428B0
:1011300073D828688003F7D50CE0FFF72DFE06462C
:1011400005E000BFFFF728FE801B6428F0D8286860
:101150008003F7D420789A4E80074FF001094FF0B2
:10116000000839D5686810F00C0F07D06868C0F324
:101170008100022809D16868C00306D42868800766
:1011800014D52069012808D110E02069B0B1C6F853
:101190000090FFF701FE074605E00AE1FFF7FCFDBE
:1011A000C01B0228C4D828688007F7D52868616961
:1011B00020F0F80040EAC10028600DE0C6F8008089
:1011C000FFF7EAFD074604E0FFF7E6FDC01B022833
:1011D00023D828688007F7D4207800072CD57948D1
:1011E000A169D9B1C0F80090FFF7D6FD074604E029
:1011F000FFF7D2FDC01B02280FD8686A8007F7D519
:1012000071484FF4FA510068B0FBF1F0009000BF54
:101210000098411E0091FAD20EE080E0C0F80080F4
:10122000FFF7BAFD074604E0FFF7B6FDC01B022832
:1012300075D8686A8007F7D42078400760D5E869D8
:101240000027C00008D4E86940F08050E861E869F0
:10125000012700F0805000905C480168C90513D454
:101260000168834641F480710160FFF795FD824675
:1012700006E000BFFFF790FDA0EB0A0064284ED8FF
:10128000DBF80000C005F5D5E06801280AD008B1F8
:10129000052813D0286A20F001002862286A20F06F
:1012A000040002E0286A40F001002862E06841F290
:1012B000883B98B1FFF770FD82460BE0286A40F04A
:1012C00004002862EEE700BFFFF766FDA0EB0A010D
:1012D00059455AD8286A8007F6D50CE0FFF75CFD1F
:1012E000824605E0FFF758FDA0EB0A0159454CD8AE
:1012F000286A8007F6D41FB1E86920F08050E861C1
:10130000E06988B36968C1F38101022944D00228E9
:10131000C6F8608004D0FFF73FFD044638E034E0B3
:10132000FFF73AFD074604E0FFF736FDC01B022831
:101330002BD828688001F7D4206AB0F5803F05D10A
:101340006868A16820F4003008436860D4E90801A7
:101350000843696821F4741108436860C6F8609016
:10136000FFF71AFD044606E025E000BFFFF714FD75
:10137000001B022809D828688001F7D51BE000BFB0
:10138000FFF70AFD001B022802D90320BDE8F88FF1
:1013900028688001F4D40EE00128F7D06868226A3A
:1013A00000F48031914204D1616A00F470108842E7
:1013B00001D00120EAE70020E8E700000010024029
:1013C00000004242800442421C00002000700040A5
:1013D00010B5401EB0F1807F01D3012010BD4FF049
:1013E000E02460610F21601701F036F90020A06150
:1013F00007202061002010BD70477047F8B50168D4
:1014000004460868CA684B6910F00F0F4FF00005DA
:1014100059D003F0010602F49077374365D0C10735
:1014200005D0D10503D5616C41F00101616441072C
:1014300005D5D90703D0616C41F0020161648107D1
:1014400005D5D90703D0616C41F00401616401073F
:1014500007D502F02001314303D0616C41F008014F
:101460006164616C00293AD0800604D5900602D5EB
:10147000204600F0BCFD20684069616CC0F380101C
:10148000090700D460B3204600F08AFD2068406957
:10149000400621D52068143050E8001F21F040019B
:1014A00040E80012002AF5D1E06BA8B16D49416314
:1014B000E06BFFF765F9002811D0E06B416B01B0DC
:1014C000BDE8F040084783060FD593060DD52046AA
:1014D000BDE8F84000F08BBD2046FFF78EFFF8BD59
:1014E0002046FFF78AFF6564F8BD266B2023012E96
:1014F0007CD1C6067AD5D60678D5086848680090AB
:1015000048694FF00206400640D5E16B0868406824
:101510000004000CE8D0A28D8242E5D9E0858869FC
:1015200020282DD020680C3050E8001F21F4807155
:1015300040E80012002AF5D12068143050E8001F5E
:1015400021F0010140E80012002AF5D12068143092
:1015500050E8001F21F0400140E80012002AF5D1B8
:1015600084F84230256320680C3050E8001F21F0D9
:10157000100140E80012002AF5D1E06BFFF7DCF81B
:101580006663A08DE18D401A81B22AE0A08DE18DC5
:10159000401A81B2E08D0028A6D00029A4D022688C
:1015A0000C3252E8000F20F4907042E80007002F40
:1015B000F5D12068143050E8002F22F0010240E8F5
:1015C0000027002FF5D184F84230256320680C30C5
:1015D00050E8002F22F0100240E80023002BF5D144
:1015E00066632046FFF708FFF8BDFFE705062BD529
:1015F000150629D594F841002128F5D1A068B0F549
:10160000805F01D12069B0B1206A411C216221684C
:1016100000784860E08C401E0004000CE084E3D1B8
:101620002068C16821F08001C1602068C16841F074
:101630004001C160D8E7206A0088C0F30800486014
:10164000206A801C2062E5E74006CDD55006CBD548
:10165000CA68204622F04002CA6084F8413000F097
:101660001EF9C1E7911F000870B5040004D094F87A
:101670004100002510B106E0012070BD84F8405003
:10168000204600F023F8242084F841002068C16837
:1016900021F40051C160204600F00AFD2068016974
:1016A00021F4904101612068416921F02A014161E2
:1016B0002068C16841F40051C1606564202084F84D
:1016C000410084F842006563002070BD30B585B0EC
:1016D00000240094019402940394006818498842FD
:1016E0002CD11848C16941F48021C161C16901F45C
:1016F00080210491816941F0080181618069124D66
:1017000000F0080004904FF48060009002200190E7
:101710000320039069462846FFF742FAE814CDE912
:101720000004694628460294FFF73AFA002211465F
:101730002720FFF79DFB2720FFF78CFB05B030BD6E
:101740000048004000100240000C01402DE9F84F15
:10175000044690F842009A4616460D46202802D0CC
:101760000220BDE8F88FB5B1AEB10020606422213F
:1017700084F842102063FFF70FFBA6858146E685BB
:10178000A0684FF480582027404501D1206920B13E
:101790002E46002529E00120E3E7002625E04B4600
:1017A000002220212046CDF800A000F0DDFC18B179
:1017B00084F842700320D4E726B1A06840451AD0CF
:1017C00038B108E020684068C0F3080025F8020B33
:1017D00008E0206978B12068406800F07F0000BF11
:1017E00006F8010BE08D401EE085E08D0028D6D183
:1017F00084F84270B5E720684068F1E770472DE94A
:10180000F843044690F84100984616460D462028B5
:1018100002D00220BDE8F88385B17EB1002060646B
:10182000212084F84100FFF7B7FAA6848146E684B8
:10183000A0682027B0F5805F02D003E00120E9E72F
:10184000206910B12E4600250EE000260CE0802114
:10185000204600F089FCA8B9C6B116F8010B216832
:101860004860E08C401EE084E08C4B464FF0000264
:10187000CDF800800028EAD14FF04001204600F06A
:1018800073FC40B184F841700320C3E735F8020BC4
:10189000C0F30800E3E784F841700020BAE770471E
:1018A000FEE70000F0B500220D4B154614460A274E
:1018B000B1FBF3F630368654B1FBF3F603FB161199
:1018C000B3FBF7F3521C861816F8016C302E00D1CA
:1018D00025B16D1C641C0A2CEAD3F0BD0022F9E787
:1018E00000CA9A3B0D4808B5816941F02001816129
:1018F000816901F020010091816941F00801816155
:10190000816901F008010091816941F00401816160
:10191000806900F00400009008BD00000010024043
:101920000C4810B50A4901604FF4E13141600021D3
:1019300081600C22C160C0E904128161C161FFF7BE
:1019400093FE002803D0BDE81040FEF7ECBC10BDAC
:101950000048004068040020FEF706FD2E4C2F4E84
:101960002F4D41F2883800276060306840682A496E
:1019700043460122491C2948FFF7E8FE607808B970
:1019800033206070C0B231281BD0322816D03328E3
:1019900019D0342823D02078401CC0B220700528EC
:1019A0000AD920A000F058FA72B66868E060A0601A
:1019B000296881F30888804726A01FE000F0D4F949
:1019C00027E000F03BF933A000F046FA72B66868F1
:1019D000E060A060296881F30888804719E06068AA
:1019E00038B10120FEF706FD08B133A006E03EA0A5
:1019F00008E00020FEF7FEFC18B143A000F02CFA2E
:101A000007E04CA000F028FA52A000F025FAFFF7FA
:101A10005FF86770A9E7000000000020680400205C
:101A20000040000853746172742070726F677261B5
:101A30006D20657865637574696F6E20666F7220BE
:101A40006D6178206572722E2E2E2E2E2E0D0A0AB2
:101A500000000000496E76616C6964204E756D620D
:101A600065722021203D3D3E20546865206E756DD5
:101A70006265722073686F756C64206265206569A9
:101A80007468657220312C20322C2033206F722034
:101A9000340D000053746172742070726F6772614C
:101AA0006D20657865637574696F6E2E2E2E2E2EEF
:101AB0002E0D0A0A000000004572726F723A20462D
:101AC0006C61736820777269746520756E2D707211
:101AD0006F74656374696F6E206661696C65642EEE
:101AE0002E2E0D0A00000000577269746520507296
:101AF0006F74656374696F6E2064697361626C658D
:101B0000642E2E2E0D0A00004572726F723A204626
:101B10006C6173682077726974652070726F746588
:101B20006374696F6E206661696C65642E2E2E0D7C
:101B30000A00000057726974652050726F74656303
:101B400074696F6E20656E61626C65642E2E2E0D59
:101B50000A00000053797374656D2077696C6C20FE
:101B60006E6F7720726573746172742E2E2E0D0A5B
:101B700000000000FEE7FEE7704700002DE9F84393
:101B800000240F460646904613460C600122694623
:101B90002848FFF7DBFD050020D19DF8000018283C
:101BA00020D006DC01280BD002280BD0042804D159
:101BB00004E0412827D0612825D0012530700DE0B0
:101BC000802401E04FF480643070221D4346B11C34
:101BD0001848FFF7BBFD050017D0002428463C60DD
:101BE000BDE8F8834346012269461248FFF7AEFD7F
:101BF00018B99DF80000182803D001259DF80000B1
:101C0000DCE70224DAE70225D8E7F178B07881F042
:101C1000FF0188420AD130190179407900EB01288F
:101C20002146301DFEF76AFB4045D7D00024012530
:101C3000D4E7000068040020704700001FB50020B2
:101C4000009001900290039003A800F0DFFA38B1F1
:101C500005281AD004281CD002281CD00FA015E09B
:101C6000164800F0F9F8164800F0F6F868460399AF
:101C7000FFF718FE13A000F0EFF8684600F0ECF84C
:101C800013A000F0E9F815A000E01AA000F0E4F8B5
:101C90001FBD28A0FAE72EA0F8E700000A0D466154
:101CA000696C656420746F20726563656976652070
:101CB0007468652066696C65210A0D00C4260008F9
:101CC000260400200A0D2053697A653A200000009E
:101CD0002042797465730D0A000000002D2D2D2D12
:101CE0002D2D2D2D2D2D2D2D2D2D2D2D2D2D2D0A47
:101CF000000000000A0A0D54686520696D6167657F
:101D00002073697A65206973206869676865722045
:101D10007468616E2074686520616C6C6F776564AF
:101D2000207370616365206D656D6F7279210A0D96
:101D3000000000000A0A0D566572696669636174E5
:101D4000696F6E206661696C6564210A0D00000090
:101D50000D0A0A41626F727465642062792075739E
:101D600065722E0A0D00000008B500208DF80000F5
:101D70000EA000F071F84FF0FF33012269461248BF
:101D8000FFF7E4FC9DF8000043280DD14FF480429A
:101D90000EA1144800F0FCFA8DF8000008B112A062
:101DA00000E01CA000F058F808BD00000A0A0D531E
:101DB000656C656374205265636569766520466964
:101DC0006C650A0D000000006804002055706C6FFF
:101DD00061646564466C617368496D6167652E6214
:101DE000696E0000004000080A0D4572726F722093
:101DF0004F63637572726564207768696C652054FF
:101E000072616E736D697474696E672046696C6582
:101E10000A0D00000A0D46696C652075706C6F61D3
:101E2000646564207375636365737366756C6C7940
:101E3000200A0D0001B5074890F84110A02902D1F1
:101E4000202180F841106423012269460148FFF7F0
:101E5000D6FC08BD68040020002201E0521C92B2AA
:101E6000815C0029FAD1014664230148FFF7C7BC11
:101E700068040020F0B5054600242A782046234651
:101E8000302A2ED16A78782A01D0582A29D1022402
:101E90001CE000BFA2F14106052E07D9A2F161079F
:101EA000052F03D91136092E04D913E0A2F130070A
:101EB000092F01D8303A04E0052E01D8373A00E066
:101EC000573A641C02EB03130B2C04D22A5D002A40
:101ED000E0D103E000202A5D002A01D101200B603F
:101EE000F0BD2A5D62B16B2A01D04B2A02D10CB140
:101EF0009B0205E06D2A01D04D2A04D11CB11B05BF
:101F000001200B600AE0A2F13006092E0CD803EB89
:101F100083036FF02F0606EB43031344641C0B2C62
:101F2000DED20128DDD1F0BD0020F0BDFEF73ABFC2
:101F300030B58FB028216846FEF77BF914210AA836
:101F4000FEF777F901210804CDE90010002402947E
:101F500002250491CDE907504FF4E010099068463E
:101F6000FFF7A6F808B172B6FEE70F20CDE90A0523
:101F70004FF48060CDE90C4002210AA80E94FEF7D0
:101F8000BBFF002801D072B6FEE70FB030BD70472E
:101F900010B5406A0021C185C184FFF72EFA10BD3B
:101FA00001680C3151E8002F22F4907241E80023BF
:101FB000002BF5D10168143151E8002F22F0010205
:101FC00041E80023002BF5D1016B012909D10168FB
:101FD0000C3151E8002F22F0100241E80023002BC1
:101FE000F5D1202180F8421000210163704708B527
:101FF00090F84210222901D0022008BD82684FF4D7
:1020000080539A4201D1016921B1816A9A421BD061
:102010004AB10AE00268816A5268C2F308020A8083
:10202000816A891C08E0026972B10268526802F094
:102030007F020A70816A491C8162C18D491E0904B0
:10204000090CC18503D01BE002685268F1E7016802
:10205000CA6822F02002CA600168CA6822F480724D
:10206000CA6001684A6922F001024A61202180F8B1
:10207000421000214163026B012A03D0FFF7BEFB2F
:10208000002008BD016301680C3151E8002F22F0E7
:10209000100241E80023002BF5D101680A68D2063E
:1020A00002D50A6849680091818DFFF7A5F9E7E735
:1020B00070B5044600680169E26821F4405111439B
:1020C00001612169A0680843616908432168CA6801
:1020D00041F20C639A430243CA6020684169A269D5
:1020E00021F44071114341611E492068884202D1A8
:1020F000FEF7A8FF01E0FEF795FF00EBC00101EB42
:102100000012606864218000B2FBF0F3B3FBF1F3CE
:102110006FF018067343B2FBF0F5B2FBF0F605EB77
:102120008305322303EB0515B5FBF1F5B6FBF1F69C
:1021300005F0F00505EB0615B2FBF0F6B2FBF0F08A
:10214000B0FBF1F06FF01802504306EB800003EB98
:102150000010B0FBF1F0216800F00F002844886007
:1021600070BD0000003801402DE9F843984617463D
:102170000D460446089E24E0701C22D0FEF70CFE9B
:10218000A0EB0800B0421AD8CEB12068C168490758
:1021900017D5802D15D0402D13D00168C9430907EC
:1021A0000FD401680025406800902046FFF7F8FE34
:1021B0000820606484F840500120BDE8F8830320C3
:1021C000FBE72068006835EA000004D00020B84230
:1021D000D2D00020F1E70120F9E700000148FFF725
:1021E0000DB900006804002041F4807141F2210221
:1021F00040004900CB0500D5401CC30300D550402A
:10220000CB03F5D580B27047FEE700002DE9F14F12
:102210000027DFF86CA188B03E46B9463C46D3465D
:10222000A6E000BF4FF0000845469DE04FF47A72EB
:1022300004A95448FFF7A2FC60B1022868D0B9F1A4
:10224000000F00D0761C052E79D91820FFF7F2FD7B
:10225000182087E00498002660B1022805D049497B
:102260008B7843450BD015207CE00620FFF7E2FD7C
:10227000022479E00620FFF7DDFD012574E0B8F1C6
:10228000000F14D082085846091DFEF78BF8E8B3FA
:102290001820FFF7CFFD1820FFF7CCFD5FF00404F6
:1022A00008F1010000F0FF084FF001095CE0087937
:1022B00068B30020344B091D02E01A54401C491C2D
:1022C0000A780AB14028F8D34FF0000C03F800C098
:1022D00060466B4601E01A54401C11F8012F202A79
:1022E00001D01028F7D303F800C006A91846FFF75D
:1022F000C1FD089844F201010068884214D91820F1
:102300000C058DF814002346012202E01EE017E0C0
:1023100022E005A91D48FFF772FA2346012205A90C
:102320001A48FFF76CFA05245046FDF7FFFF08989E
:10233000069901600620FFF77DFD432009E010E0CB
:102340000620FFF777FD01252F460DE004990620B2
:102350008B44FFF76FFDA3E71820FFF76BFD1820F4
:1023600084E74320FFF766FD55EA04003FF45EAFC3
:1023700057EA04003FF456AF09B02046BDE8F08F9D
:1023800000400008200000202604002068040020EF
:102390002DE9F74F86B04FF0000A0120AC4E0190B6
:1023A00001220898727086F802A0FF23D046554695
:1023B0005746F370544604E006EB040C641C8CF89A
:1023C00004300B5D0BB1402CF6D332190021117192
:1023D000014602A8FFF766FA02A8641D02E0315523
:1023E000641C7F1CC15D0029F9D14FF48019DFF80E
:1023F00060B202E000203055641C842CFAD31FE048
:102400005C464E464B468322611C9248FFF7F7F923
:102410008021201DFDF772FF0446000AFFF70AFD28
:10242000E0B2FFF707FD3346012269468948FFF70E
:102430008DF960B10AF1010ABAF1050F00D3012547
:1024400058EA0500DCD006980290089C7CE09DF8D4
:102450000000062815D01828EED13346012269461F
:102460007C48FFF773F90028E6D19DF80000182892
:10247000E2D10220FEF71CFA764800684068022587
:10248000DAE74FF00108D7E7DDE90103704AC6B289
:102490004FF480672046BC4201D3394600E08021DA
:1024A000884200D30846B1F5806F07D001275770E6
:1024B0009670F643D6700426071D06E00227F6E75D
:1024C00013F801CB02F806C0761CBE42F8D388424E
:1024D00007D81A23001D091D01E01354401C88422F
:1024E000FBD34FF0000A8DF800A0574629E000BF4B
:1024F0004FF48066B44200D28026F21C4B46D84688
:102500000BF101015348FFF77AF9314608F1040055
:10251000FDF7F4FE8046000AFFF78CFC08F0FF0090
:10252000FFF788FC4B46012269464A48FFF70EF93F
:1025300018B99DF80000062811D07F1C052F00D384
:1025400001255AEA0500D3D00CB1002D9CD00024FF
:1025500026468DF800402746DFF8F8801FE00298F5
:102560004FF0010A3044B442029008D90198A41BEC
:10257000102802D0401C0190E0E70525DEE700248A
:10258000DCE70420FFF756FC4B4601226946314840
:10259000FFF7DCF840B17F1C052F00D3012554EA7A
:1025A0000500EED0E5B14EE09DF80000062815D0FC
:1025B0001828F1D14B46012269462648FFF7C6F894
:1025C0000028E9D19DF800001828E5D10220FEF787
:1025D0006FF9D8F8000040680225DDE70124DBE749
:1025E00001208BF801008BF80260FF208BF80300BC
:1025F0005C4604202654401CC0B28428FAD34E46C0
:102600004B468322611C1348FFF7F9F88021201DF7
:10261000FDF774FE0446000AFFF70CFCE0B2FFF77A
:1026200009FC3346012269460A48FFF78FF850B982
:102630009DF80000182806D10220FEF739F9D8F8D5
:1026400000004068022509B02846BDE8F08F000070
:1026500020000020680400200907090E002804DB80
:1026600000F1E02080F80014704700F00F0000F146
:10267000E02080F8141D7047FEF79CFBFFF758FC24
:1026800040F6B830FEF714F9FFF72CF9FFF748F9D8
:10269000FDF77CFEFFF760F9FEE701020203040587
:1026A000060708090A0B0C0D0E0F101000000000A1
:1026B00000000000010203040607080900000000F2
:1026C000010203040A0A0D2050726F6772616D6D7A
:1026D000696E6720436F6D706C6574656420537517
:1026E000636365737366756C6C79210A0D2D2D2DEE
:1026F0002D2D2D2D2D2D2D2D2D2D2D2D2D2D2D2D0A
:102700002D2D2D2D2D2D2D2D2D2D2D2D2D0D0A2049
:102710004E616D653A200000382700080000002057
:10272000200000006C01000858270008200000204D
:10273000100B0000880100080000000000000000ED
:102740000000000000000000010000001000000078
:082750000000000000127A00F5
:0400000508000131BD
:00000001FF
